:02000000040AF0
:080008009F0C0200080C060029
:10001000000C2600490A380C2800070C26000000B6
:1000200000000000000000000000000000000000D0
:100030000000000C2600000000000000000000008E
:10004000000000000000E8020D0A0008100C290062
:10005000070C260000000000000000000000000067
:100060000000000000000000000C2600000000005E
:10007000000000000000000000000000E902280A63
:100080000008410C2700000000000000E702430ABE
:1000900000080B09410926092609410926094109D9
:1000A0004109260926094109260941094109490A48
:021FFE00E90FE9
:00000001FF
